:020000040000FA
:020000000428D2
:08000800FF30A200FF30A3004D
:10001000FF30A400FF30A5000F30A600A901AA01FF
:1000200024138A150A12D221A4178A150A12CF2185
:100030008A150A120022203098000D3099008A1586
:100040000A120322903098001A081A081A08003081
:100050009900F801FE01FC01FA01F701FD01FB0125
:10006000F901FF308A150A12EB218A150A12712054
:1000700023108A150A12E121A3108A150A12DE2123
:1000800023118A150A12DB21A3118A150A12D8211D
:1000900023128A150A12D521A2148A150A12E42104
:1000A00027128A150A12B62127148A150A12C221AC
:1000B000A7108A150A12BF2127118A150A12BC211E
:1000C000A7118A150A12B92101308A150A12402196
:1000D00027108A150A12C221A7148A150A12BF21F5
:1000E00027118A150A12BC21A7118A150A12B921F3
:1000F00001308A150A12402127108A150A12C221DE
:10010000A7108A150A12BF2127158A150A12BC21C9
:10011000A7118A150A12B92101308A150A12402145
:1001200027108A150A12C221A7108A150A12BF21A8
:1001300027118A150A12BC21A7158A150A12B9219E
:1001400001308A150A124021A7118A150A12B92115
:100150008A150A129F208A150A127F2002308A15FA
:100160000A1279204F308A150A12CA204E308A1599
:100170000A12CA2034308A150A12CA2049308A1558
:100180000A12CA2059308A150A12CA2020308A154C
:100190000A12CA2032308A150A12CA2030308A1553
:1001A0000A12CA2030308A150A12CA2035308A1540
:1001B0000A12CA2040308A150A12792052308A1554
:1001C0000A12CA204F308A150A12CA2056308A15E0
:1001D0000A12CA2045308A150A12CA2052308A15DE
:1001E0000A12CA2042308A150A12CA204F308A15D4
:1001F0000A12CA2058308A150A12CA2020308A15DD
:100200000A12CA2076308A150A12CA2032308A159C
:100210000A12CA2032308A150A12CA2020308A15E2
:100220000A12CA2020308A150A12CA2044308A15C0
:100230000A12CA2057308A150A12CA2001308A15BC
:100240000A12372101308A150A12372120118A112A
:100250000A12851C2C2920158A110A12201D7B29BF
:100260008A150A127F2040308A150A127920203020
:100270008A150A12CA2020308A150A12CA2045306F
:100280008A150A12CA2058308A150A12CA2050301C
:100290008A150A12CA2045308A150A12CA2052301D
:1002A0008A150A12CA2049308A150A12CA204D300E
:1002B0008A150A12CA2045308A150A12CA204E3001
:1002C0008A150A12CA2054308A150A12CA204130EF
:1002D0008A150A12CA204C308A150A12CA20203008
:1002E0008A150A12CA2020308A150A12CA20013043
:1002F0008A150A12372127148A150A12C2218A1573
:100300000A127F20B101CB01A011A0148A110A1298
:10031000A0198E298A110A12A01891298A110A128D
:10032000F2298A110A12B9275208AB0000308A1547
:100330000A1279202B08243C8A110A120319A429D5
:100340008A110A12A018A7298A110A12AF298A1144
:100350000A12B9275208AB008A110A129A298A1187
:100360000A12A01CEF298A150A1226205208AB0097
:100370008A150A1226205208AC008A150A12262075
:100380005208AD008A150A1226205208AE008A15BE
:100390000A1226205208AF002E084D3C8A110A127C
:1003A000031DEE292F08433C8A110A12031DEE2972
:1003B0002D08523C8A110A12031DEE292C08503CCC
:1003C0008A110A12031DEE292B08473C8A110A12D2
:1003D000031DEE29A0158A110A12EF29A0118A1116
:1003E0000A1286298A110A12A01C0E2A8A150A12DC
:1003F00026205208AB0040307D028A110A12031CED
:10040000042A8A110A120E2A8A150A122620520874
:100410008A150A1216208A110A12FB298A110A1259
:10042000A01C1E2E8A110A12A01D1E2E8A150A1249
:1004300007205408B4008A150A1207205408B50092
:100440008A150A1207205408B6008A150A120720D6
:100450005408B7008A150A1207205408B8008A15F4
:100460000A1207205408B9000230B90730303902A7
:10047000093C8A110A120318412A0A303902B900CC
:10048000B80A30303802053C8A110A1203184B2A88
:100490003030B800B70A30303702093C8A110A12EE
:1004A0000318562A0A303702B700B60A303036022F
:1004B000053C8A110A120318602A3030B600B50ACA
:1004C0008A150A12072054082C3C8A110A120319B3
:1004D0006C2A8A110A12602A8A150A120720540807
:1004E000413C8A110A12031D792A20168A110A1228
:1004F0007A2A20128A150A12072054082C3C8A11E5
:100500000A120319862A8A110A127A2A8A150A12ED
:1005100007205408C0008A150A1207205408C10099
:100520008A150A1207205408C2008A150A120720E9
:100530005408C3008A150A1207205408C4008A15FB
:100540000A1207205408C4008A150A12072054080A
:100550002C3C8A110A120319B02A8A110A12A42A01
:100560008A150A12072054082C3C8A110A12031912
:10057000BC2A8A110A12B02A8A150A1207205408C6
:10058000C5008A150A1207205408C6008A150A12E7
:1005900007205408C7008A150A1207205408C8000B
:1005A0008A150A1207205408C9008A150A12072062
:1005B00054082C3C8A110A120319E12A8A110A12E2
:1005C000D52A8A150A1207205408CA008A150A1269
:1005D000072054082C3C8A110A120319F22A8A11A6
:1005E0000A12E62A8A150A12072054082C3C8A119E
:1005F0000A120319FE2A8A110A12F22A8A150A120D
:10060000072054082C3C8A110A1203190A2B8A115C
:100610000A12FE2A8A150A1207205408BA008A15FF
:100620000A1207205408BB008A150A120720540832
:10063000BC008A150A1207205408BD008A150A1248
:1006400007205408BE008A150A1207205408BF006C
:100650004A08453C8A110A12031D562B30304502C8
:10066000EB006430EC008A150A124A22D4005408C8
:10067000D30030304702D50030304602EB000A305C
:10068000EC008A150A124A22D6005608550753076D
:10069000E9001430EA008A150A123122D200520809
:1006A000093E413EAB008A110A127B2B30304502D5
:1006B000EB006430EC008A150A124A22D90059086E
:1006C000D80030304702DA0030304602EB000A3002
:1006D000EC008A150A124A22DB005B085A07580709
:1006E000E9001430EA008A150A123122D7005708AF
:1006F000083C413EAB0030304102D800303040026F
:10070000EB000A30EC008A150A124A22D900590877
:100710005807E9000A30EA008A150A123122D70088
:100720005708093E413EAC004A08453C8A110A126E
:10073000031DC92B30304502EB006430EC008A15F4
:100740000A124A22DD005D08DC0030304702DE007C
:1007500030304602EB000A30EC008A150A124A22B9
:10076000DF005F085E075C07E9001430EA008A15C5
:100770000A121A22DB005B08E6000130E7008A1546
:100780000A120622DA005A08303EAD008A110A1217
:10079000F62B30304502EB006430EC008A150A126B
:1007A0004A22E3006308E20030304702E4003030C0
:1007B0004602EB000A30EC008A150A124A22E500D4
:1007C000650864076207E9001430EA008A150A1216
:1007D0001A22E1006108E6000130E7008A150A12DA
:1007E0000622E0006008093C303EAD004108AE0042
:1007F0004A08453C8A110A12031D3B2C303047023F
:100800000139003C8A110A12031D202C30304902A4
:10081000E10030304802EB000A30EC008A150A1281
:100820004A22E20062086107E9000530EA008A1501
:100830000A123122E0006008B3008A110A12382C33
:1008400030304902E40030304802EB000A30EC005E
:100850008A150A124A22E500650864073C3EE90051
:100860000530EA008A150A123122E3006308B3005A
:100870008A110A12762C303047020139013C8A1164
:100880000A12031D5E2C30304902E4003030480269
:10089000EB000A30EC008A150A124A22E5006508CE
:1008A0006407E9000530EA008A150A123122E300E4
:1008B00063080B3CB3008A110A12762C30304902CF
:1008C000E70030304802EB000A30EC008A150A12CB
:1008D0004A22E80068086707E9000530EA008A153F
:1008E0000A123122E6006608173CB3003308203EA6
:1008F000413EAF0030304302E40030304202EB00B2
:100900000A30EC008A150A124A22E50065086407DD
:10091000E9000530EA008A150A123122E300630873
:10092000B0000310300D413EB00030304302E7000C
:1009300030304202EB000A30EC008A150A124A22DB
:10094000E80068086707E9000530EA008A150A121E
:100950001A22E6006608B3003308023C8A110A1224
:100960000318B32CB00A3308023C8A110A12031D83
:10097000C02C4408053C8A110A120318C02CB00A86
:100980002030B00740308A150A12792034088A15C1
:100990000A12CA2035088A150A12CA203A308A1566
:1009A0000A12CA2036088A150A12CA2037088A1580
:1009B0000A12CA203A308A150A12CA2038088A1543
:1009C0000A12CA2039088A150A12CA2020308A154C
:1009D0000A12CA2020308A150A12CA208A110A1265
:1009E00020190D2D2B088A150A12CA202C088A15E9
:1009F0000A12CA202D088A150A12CA202E088A1542
:100A00000A12CA202F088A150A12CA2030088A152D
:100A10000A12CA208A110A12892DCB088A110A12D9
:100A2000031D2D2D2B088A150A12CA202C088A15A1
:100A30000A12CA202D088A150A12CA202E088A1501
:100A40000A12CA202F088A150A12CA2030088A15ED
:100A50000A12CA208A110A12892DB1088A110A12B3
:100A6000031D4A2D2B088A150A12CA202C088A1544
:100A70000A12CA202D088A150A12CA202E088A15C1
:100A80000A12CA202F088A150A12CA2030088A15AD
:100A90000A12CA203108013C8A110A12031D682D6E
:100AA0004C088A150A12CA204D088A150A12CA2053
:100AB00020308A150A12CA2053308A150A12CA2019
:100AC00041308A150A12CA2054308A150A12CA20E7
:100AD0003108023C8A110A12031D882D20308A1524
:100AE0000A12CA204E088A150A12CA204F088A150F
:100AF0000A12CA2050088A150A12CA2051088A15FB
:100B00000A12CA206D308A150A12CA20FF30B100BD
:100B1000B10A00308A150A1279203A088A150A1299
:100B2000CA203B088A150A12CA202F308A150A12D9
:100B3000CA203C088A150A12CA203D088A150A12E2
:100B4000CA20303037020139013C8A110A12031DD4
:100B5000C02D20308A150A12CA204F308A150A1279
:100B6000CA2044308A150A12CA2044308A150A1253
:100B7000CA2020308A150A12CA208A110A12D42DDE
:100B800020308A150A12CA2045308A150A12CA2056
:100B900056308A150A12CA2045308A150A12CA2010
:100BA0004E308A150A12CA208A110A12201EFB2D05
:100BB00027158A150A12BC21A7118A150A12B92114
:100BC0000B308A150A12792036088A150A12CA20B3
:100BD00037088A150A12CA203A308A150A12CA2022
:100BE00038088A150A12CA2039088A150A12CA203A
:100BF0008A110A121B2E27118A150A12BC21A71569
:100C00008A150A12B9210B308A150A127920493047
:100C10008A150A12CA204E308A150A12CA20563086
:100C20008A150A12CA2041308A150A12CA204C308D
:100C30008A150A12CA208A110A12462E8A110A122D
:100C4000A018462E48308A150A1279204E308A158F
:100C50000A12CA204F308A150A12CA2020308A157B
:100C60000A12CA2047308A150A12CA2050308A1543
:100C70000A12CA2053308A150A12CA2020308A1557
:100C80000A12CA2020308A150A12CA20FD01FE016C
:100C9000A7148A150A12BF2101308A150A124921A8
:100CA000A7108A150A12BF21B1088A110A12031D62
:100CB000B32F8A110A12201DB32FA011A0148A117C
:100CC0000A12A019672E8A110A12A0186A2E8A1118
:100CD0000A12C72E8A110A12B9275208AB002B0834
:100CE000243C8A110A120319792E8A110A12A018BB
:100CF0007C2E8A110A12842E8A110A12B9275208F0
:100D0000AB008A110A126F2E8A110A12A01CC42E7F
:100D10008A150A1226205208AB008A150A122620CC
:100D20005208AC008A150A1226205208AD008A1516
:100D30000A1226205208AE008A150A1226205208EE
:100D4000AF002E08473C8A110A12031DC32E2F083C
:100D5000413C8A110A12031DC32E2D08473C8A11FB
:100D60000A12031DC32E2C08503C8A110A12031DBF
:100D7000C32E2B08473C8A110A12031DC32EA0154F
:100D80008A110A12C42EA0118A110A125F2E8A112A
:100D90000A12A01CE32E8A150A1226205208AB0064
:100DA00040307D028A110A12031CD92E8A110A12C0
:100DB000E32E8A150A12262052088A150A121620D6
:100DC0008A110A12D02E8A110A12A01C812F8A11B0
:100DD0000A12A01D812FB201053032028A110A12B7
:100DE000031CF52E8A110A12052F8A150A120720F4
:100DF00054082C3C8A110A120319012F8A110A1275
:100E0000F52EB20A8A110A12EC2E8A150A12072050
:100E10005408D20030305202CB008A150A12072043
:100E20005408CC008A150A1207205408CC008A15F1
:100E30000A1207205408CD00CB088A110A120319A0
:100E40007E2F8A150A1207205408CE008A150A122E
:100E5000072054082C3C8A110A120319322F8A11D8
:100E60000A12262F8A150A1207205408CE008A1566
:100E70000A1207205408CF008A150A1207205408C6
:100E8000D0008A150A1207205408D1004E082E3CC3
:100E90008A110A12031D542F2030D1002030D000B7
:100EA0002030CF002030CE004F082E3C8A110A128D
:100EB000031D622F4E08D1002030D0002030CF001B
:100EC0002030CE0050082E3C8A110A12031D702FCC
:100ED0004F08D1004E08D0002030CF002030CE0087
:100EE00051082E3C8A110A12031D7E2F5008D10092
:100EF0004F08D0004E08CF002030CE008A110A12D1
:100F0000A52F8A110A12A018A52F48308A150A1297
:100F100079204E308A150A12CA204F308A150A12DB
:100F2000CA2047308A150A12CA2050308A150A1280
:100F3000CA2053308A150A12CA2020308A150A1294
:100F4000CA2020308A150A12CA20FD01FE01271688
:100F50008A150A12B62101308A150A124921271270
:100F60008A150A12B6218A110A1284298A110A12D4
:100F7000B62FD200FF30D300FF30D4008A150A12FA
:100F800045205508D2008A110A12201FCE2FA01426
:100F90008A150A1206288A110A12CF2FA010D30828
:100FA0008A110A120319D82F8A110A12A01CDB2FEA
:100FB0008A150A120628D4088A110A120319E42F86
:100FC0008A110A12A01CE72F8A110A12FE2F013083
:100FD0005402D4008A150A1245205508D2008A11FD
:100FE0000A12201FFA2FA0148A150A1206288A1145
:100FF0000A12FB2FA0108A110A12DB2F01305302B4
:10100000D300FF30D4008A110A12CF2F08004F30CE
:101010007E028A150A12031C0E28FE017E08A03EDD
:1010200084008313FE0A0008D4000800D3004F3068
:101030007D028A150A12031C1E28FD017D08A03EB0
:101040008400831353088000FD0A0800D20098181A
:10105000342818193E288C1E27288B138B1B2D280B
:101060001A088B17D20044288B138B1B34281812B4
:101070001A081A081A0818168B1727288B138B1BA7
:101080003E281A088B1727280800D5008A150A124F
:101090008C1E4E28A0178A150A124F28A0139818E4
:1010A0005A28181964288B138B1B53281A088B177E
:1010B000D5006A288B138B1B5A2818121A081A0895
:1010C0001A0818168B174F288B138B1B64281A08C5
:1010D0008B174F2820138A150A12A01F702820177B
:1010E00008008A150A12002287309F008A150A120A
:1010F000032AE9006908803E8A150A12D8280830B8
:101100008A150A12D82001308A150A12D820C83050
:101110008A150A127E2102308A150A12D820C83098
:101120008A150A127E2106308A150A12D8200C3040
:101130008A150A12D820C8308A150A127E298A1503
:101140000A122F2164308A150A125221A8108A151A
:101150000A12B32103308A150A12EE2032308A15A2
:101160000A12922103308A150A12EE2032308A15B3
:101170000A12922103308A150A12EE2032308A15A3
:101180000A12922132308A150A12D82028308A1584
:101190000A12D828E900A8148A150A12B321690E88
:1011A0000F398A150A12EE2069088A150A12EE28EC
:1011B000EA00A8108A150A12B3216A0E0F398A159F
:1011C0000A12EE2082308A150A125B216A088A15FB
:1011D0000A12EE2082308A150A125B29EB002811D0
:1011E0008A150A12B021A8158A150A12AD212812F3
:1011F0006B080139003C8A150A12031800292816C9
:101200008A150A12AA21A8126B080239003C8A1515
:101210000A1203180C29A8168A150A12A7212813E6
:101220006B080439003C8A150A120318182928177C
:101230008A150A12A421A8136B080839003C8A15E4
:101240000A1203182429A8178A150A12A121A81125
:101250008A150A12AD21FA308A150A127E29003049
:101260008A150A12E72100308A150A12C529AB0037
:101270002B08EC006430ED0064308A150A126429F2
:10128000AB002B08EC006430ED0014308A150A1214
:101290006429D2005208EC006430ED000A308A154F
:1012A0000A126429AB002B08EC000A30ED00013073
:1012B0008A150A126429EB006B08EC000130ED007E
:1012C00001308A150A126429EE00FF30EF006D0824
:1012D000F1006C08F00017308A150A126F07031826
:1012E0006E298A150A12F00B6B298A150A12F10B66
:1012F00069298A150A12EE0B67290800EC006C08B0
:10130000ED00ED088A150A12031D89298A150A12B3
:1013100091290A308A150A129221ED038A150A12C0
:1013200081290800EE00F430EF00FC30F0008A154F
:101330000A126E086F07031C0034700703189D29FA
:1013400008008A150A12C9298A150A12C9298A159C
:101350000A12C9298A150A12C9298A150A12C92925
:101360008A150A12C9298A150A12C9298A150A1268
:10137000CC298A150A12CC298A150A12CC298A1579
:101380000A12CC298A150A12CC29A8008A150A1239
:10139000C9292808880008002708860008008A153F
:1013A0000A12F7298A150A12F7298A150A12FA2948
:1013B0008A150A12FA298A150A12FA298A150A12B6
:1013C000FA298A150A12FA298A150A12FD29A50096
:1013D0008A150A12EF29A2008A150A12FD2925088A
:1013E0008A150A12002288008A150A12032A240884
:1013F000670008002308660008002208650008004E
:10140000831603130800831203130800E70067081C
:10141000003C8A150A12031C102A8A150A12182A7F
:101420000310E60C01306702E7008A150A12072A4A
:1014300066080800EA00EA088A150A1203192F2A2A
:101440006A0869028A150A120318292A8A150A12DB
:101450002F2A6A086902E9008A150A12202A6908F7
:101460000800EA00EB01EA088A150A120319482A63
:101470006A0869028A150A120318412A8A150A1293
:10148000482A6A086902E900EB0A8A150A12382A12
:101490006B080800EC00ED016C08003C8A150A128C
:1014A000031C552A8A150A125D2A6B08ED070130C4
:0E14B0006C02EC008A150A124C2A6D08080026
:02400E00723FFF
:00000001FF
